:020000040800F2
:10000000600700246D030008B927000801270008D5
:10001000B127000881040008392D00080000000005
:10002000000000000000000000000000392A000865
:100030008904000800000000F1270008412A000898
:100040008B0300088B0300088B0300088B03000858
:100050008B0300088B0300088B0300088B03000848
:100060008B0300088B0300088B0300088B03000838
:100070008B0300088B0300088B0300088B03000828
:100080008B0300088B0300088B030008C1040008E1
:100090008B0300088B0300088B0300088B03000808
:1000A0008B0300088B0300088B0300088B030008F8
:1000B000C92B00088B0300088B0300088B03000882
:1000C0008B0300088B0300088B0300088B030008D8
:1000D0008B0300088B0300088B0300088B030008C8
:1000E0008B0300088B030008000000008B0300084E
:1000F0008B0300088B0300088B0300088B030008A8
:100100008B0300088B0300088B0300088B03000897
:100110008B0300088B0300088B0300088B03000887
:100120008B0300088B0300088B0300088B03000877
:100130008B0300088B0300088B0300088B03000867
:1001400000000000000000000000000000000000AF
:100150008B0300088B0300088B0300088B03000847
:100160008B0300088B0300088B0300088B03000837
:100170008B0300088B0300088B03000800000000BD
:100180008B0300088B0300088B0300088B03000817
:100190008B0300088B0300088B0300088B03000807
:1001A0008B0300088B0300088B030008000000008D
:1001B0008B0300088B0300088B0300088B030008E7
:1001C0008B0300088B030008000000000000000003
:1001D00000000000000000008B0300080000000089
:1001E000000000000000000000000000000000000F
:1001F00000000000000000008B0300088B030008D3
:100200008B0300088B030008000000008B0300082C
:100210008B0300088B0300088B0300088B03000886
:100220008B030008000000008B03000800000000A2
:100230008B0300088B030008000000008B030008FC
:100240008B0300088B0300088B0300088B03000856
:100250008B0300088B0300088B0300088B03000846
:100260008B0300088B0300088B0300088B03000836
:100270008B0300088B0300088B03000800000000BC
:100280008B0300088B0300088B0300088B03000816
:10029000000000008B0300088B0300080000000032
:1002A000000000008B0300088B0300088B0300088C
:1002B0008B0300088B0300088B0300088B030008E6
:1002C0008B0300088B0300088B03000800F002F882
:1002D00000F03CF80AA090E8000C82448344AAF1A4
:1002E0000107DA4501D100F031F8AFF2090EBAE8A2
:1002F0000F0013F0010F18BFFB1A43F0010318475A
:10030000402B0000602B0000103A24BF78C878C151
:10031000FAD8520724BF30C830C144BF04680C600B
:10032000704700000023002400250026103A28BF53
:1003300078C1FBD8520728BF30C148BF0B60704757
:100340001FB502F042FD1FBD10B510BD00F05CF8F6
:100350001146FFF7F5FF02F02FFD00F07AF803B425
:10036000FFF7F2FF03BC00F081F800000A48804765
:100370000A4880470A480047FEE7FEE7FEE7FEE737
:10038000FEE7FEE7FEE7FEE7FEE7FEE70548064973
:10039000064A074B70470000A1040008F12A000834
:1003A000CD020008600100246007002460030024DF
:1003B000600300244FF0000200B5134694469646B1
:1003C000203922BFA0E80C50A0E80C50B1F1200168
:1003D000BFF4F7AF090728BFA0E80C5048BF0CC016
:1003E0005DF804EB890028BF40F8042B08BF704774
:1003F00048BF20F8022B11F0804F18BF00F8012BE6
:100400007047704770477047754600F02BF8AE464E
:1004100005006946534620F00700854618B020B510
:10042000FFF7B4FFBDE820404FF000064FF0000793
:100430004FF000084FF0000BAC46ACE8C009ACE848
:10044000C009ACE8C009ACE8C00921F007018D463D
:10045000704710B50446AFF300802046BDE8104059
:10046000FFF77DBF004870471000002401491820A5
:10047000ABBEFEE72600020070470000000000004F
:10048000FEE70000000000007047000000000000D0
:10049000EFF3108072B600BFFEE70000000000001E
:1004A00044F60C00C5F60200016841F0020101604B
:1004B00050F8081C8904FBD57047000000000000BC
:1004C00080B540F27000C2F2004000F0F5F880BD47
:1004D0002DE9F04F82B00168C76BD0E90DA2D1F8C9
:1004E00084304FF6FC74A34343EA8A03C1F8843096
:1004F000D1F88430019223F47F0343EA0243C1F828
:10050000843002EB0A03D1F888406FF38F0444EA89
:100510008304C1F88840D1F88840009724F4FE0491
:1005200044EA0744C1F8884003EB4704D1F8A030FF
:100530006FF38F0343EA8403C1F8A030D1F8A050D1
:10054000D0F840B025F4FE0545EA0B45C1F8A050AF
:10055000D0F84480D1F8B0506FF38F0508FB0B44FE
:1005600008FB0BF845EA8405C1F8B050D1F8B0603B
:10057000856C26F4FE0646EA0546C1F8B060D0F860
:100580004C9009FB0547D1F8AC406FF38F0409FB91
:1005900005F944EA8704C1F8AC40D0E9144606FBEB
:1005A0000472D1F8F0706FF38F0747EA8207C1F841
:1005B000F070D1F8F030876D23F47C1343EA0743E1
:1005C000C1F8F03002EB4702D1F8C0306FF38F036F
:1005D00043EA8202C1F8C020D1F8C020C36D22F4E2
:1005E0007C1242EA0342C1F8C0204AF60042D1F828
:1005F000C0C0D0F860E0C4F20002019D02EB8A02A4
:100600002CF07C5C06FB04FA009C4CEA0E6C02EBBE
:100610008505C1F8C0C005EBC406846E06EB8801F1
:10062000056701EB890C63430CEB8A05C266C0E9E0
:100630001E1C0EFB04F105EBC70707EB8303C0F894
:1006400084704DF2FC37466703EB8101C4F200076A
:10065000B942C0F88050C0F88830C0F890100AD96C
:10066000D0F89C1041F02001C0F89C10032180F8C4
:10067000981001210CE0D0F890108A4207D2002196
:1006800042F8041BD0F890309A42F9D300E00021E0
:10069000084602B0BDE8F08F70470000000000007F
:1006A00070470000000000007047000000000000DC
:1006B00070470000000000002DE9F04F87B00446AD
:1006C0004AF61000C4F2000001684AF61400C4F2B1
:1006D00000000268206802EA010A056DD0F8549013
:1006E000076DD0F85480036D0293436D0193036D41
:1006F0000693436D0593036D0493436D0393436D1C
:10070000066D06EA030B5FEACB530BD54FF48071FD
:1007100001654AF610010020C4F20001086020467D
:10072000FFF7C6FF05EA09064AF610095FEA4B50D3
:10073000C4F200094FEA8A750ED52068D0F8DC10A3
:10074000D0F8E42011404FF4806202650020C9F81F
:100750000000204600F0B0FA08EA070806F47046E8
:1007600055B12068002101650AF00300C9F80000B6
:1007700020462946FFF790FFDDE9011000EA010756
:1007800008F00F0546B12068314606650020C9F81B
:100790000000204600F098FA07F0F00645B1206806
:1007A000294605650020C9F80000204600F064FADB
:1007B00046B12068314606650020C9F80000204691
:1007C00000F05EFA5FEA0B5000F1BF805FEA8B50E9
:1007D00000F1C9805FEA0B3000F1D8805FEACB30CE
:1007E00009D520684FF4803101650020C9F8000068
:1007F000204600F05DFA5FEA4B30DDE9031000EAC5
:10080000010509D520684FF4802101650020C9F851
:100810000000204600F048FA5FEA8B30DDE9051061
:1008200000EA010005F060710CD522684FF4003336
:1008300013650022C9F80020D4F89C2042F0800201
:10084000C4F89C2000F0715539B120680165002082
:10085000C9F800002046FFF727FF4DB12068056565
:100860000020C9F80000D4F89C002843C4F89C007C
:100870002068A9F5016188425ED1606881688907B6
:100880005AD0016A426A036A476A114003EA0702C2
:1008900002F03005D0F82080D0F82490026A04924B
:1008A00011F00F01D0F824B0026A0692426A059254
:1008B000466AD0F820A003D00162204600F0E8F993
:1008C00008EA09072DB1606829460562204600F054
:1008D000E7F906EA0A0007F4C0754006049800EA42
:1008E0000B060AD560684023C16BC26B090C02F08D
:1008F0003F020362204600F0CFF9DDE9051000EA6F
:10090000010706F4FC462DB16068294605622046C1
:1009100000F0BAF907F4F02036B161680E62D4F83D
:100920009C103143C4F89C1030B161680862D4F85F
:100930009C100843C4F89C00D4F89C0010B12046D9
:10094000FFF7AEFE07B0BDE8F08F20684FF40061FE
:1009500001650020C9F80000204600F0B9F95FEAFF
:100960008B507FF537AF2068D0F8D810D0F8E02052
:1009700011404FF4007202650020C9F800002046C3
:1009800000F09EF95FEA0B307FF528AF20684FF446
:10099000002101650020C9F80000204600F068F938
:1009A0005FEACB303FF51DAF25E7000000000000F7
:1009B0002DE9F04130B34AF200080446C4F20008C1
:1009C0000068404502D108F58070606094F8980096
:1009D00028B9002084F89900204600F0F5F8206836
:1009E000816921F01001816100F046FA054600BFDF
:1009F00020688169090708D500F03EFA401B0B28E2
:100A0000F6D312E00120BDE8F081816941F00101D7
:100A1000816100F031FA054620688169C90710D16B
:100A200000F02AFA401B0B28F6D3D4F89C0040F0C3
:100A30000100C4F89C00032084F898000120BDE860
:100A4000F081816941F002018161217C826922F09B
:100A50004002012918BF40328261617C826922F420
:100A60008042012908BF02F580428261A17C82692F
:100A700022F48052012918BF02F5805282618169F7
:100A800021F44073D4E902120B438361836923F09C
:100A9000A4038361036923F010030361AAB1022A4E
:100AA0000FD0012A03D1826942F004020CE083696D
:100AB000032A43F080038361036943F0100202615B
:100AC00003D1826942F020028261D4E90552E369D0
:100AD000561E6FF0FF02276A02EB0323013F43EA31
:100AE0004663B1F5407F47EA030740F20003CFF6C3
:100AF000FF7303EB054647EA0601C16110D1D4E953
:100B00000B65D4E90917013F02EB06226FF00F06CF
:100B10003A4306EB05173A4303EB01411143C16029
:100B2000216E29B1626ED0F8C0301A43C0F8C020DF
:100B3000E26DCA4242F6E451C0F6000109D0D0F895
:100B4000C820A36E22F0070251F823301A43C0F8E0
:100B5000C820226C4AB1D0F8BC20636C22F0070296
:100B600051F823301A43C0F8BC20A26C52B1D0F81F
:100B7000BC20E36C22F0700251F8233042EA0312E9
:100B8000C0F8BC20226D52B1D0F8BC20636D22F4B5
:100B9000E06251F8231042EA0121C0F8BC10404540
:100BA00004D16068816821F0030181600020C4F8ED
:100BB0009400C4F89C00012084F898002046FFF7B8
:100BC00087FCBDE8F0810000B0B5B6B0044602A8CD
:100BD000B8210025CDE93455CDE932553195FFF7DF
:100BE000E9FB4AF200012068C4F20001884201D00A
:100BF00036B0B0BD4FF4004002904FF080501D90D1
:100C000002A8039500F020FA08B1FFF741FC44F276
:100C1000E040C5F60200C16841F48071C160C1685E
:100C200001F4807101910199016841F008010160AE
:100C3000006831A900F0080001900198032031906C
:100C4000022032900020CDE933000920359040F693
:100C50000040C5F6020000F03FF8132000210022FA
:100C600000F0BAF9132000F0B3F936B0B0BD0000BF
:100C70007047000000000000704700000000000006
:100C800070470000000000007047000000000000F6
:100C900070470000000000007047000000000000E6
:100CA00070470000000000007047000000000000D6
:100CB00070470000000000007047000000000000C6
:100CC00070470000000000007047000000000000B6
:100CD00070470000000000002DE9F04F83B00C6861
:100CE000002C00F0C68000F1264242F2004702F1DB
:100CF000FF72C5F602074FEAB22201920A22B842F9
:100D000008BF0922002500274FF0010A009209E0E0
:100D10000C68043734FA0AF20AF1010A05F10205F7
:100D200000F0A780AAF10109012202FA09FE14EAE3
:100D30000E08EDD0D1F804B00BF00304A4F1010CBF
:100D4000BCF1010F11D803228668AA40CB6826EABD
:100D50000202AB401A438260CBF30013426822EADE
:100D60000E0203FA09F31A434260032C1ED0032338
:100D7000C268AB40022C22EA03028B6803FA05F337
:100D800042EA0302C26011D16FF0030207F01C06B1
:100D900002EA59020F23024403FA06F4D2F820C0F3
:100DA0000B692CEA0404B340234313620323026853
:100DB000AB404E689A4306F00303AB4016F4403F45
:100DC00042EA03020260A3D044F2F44340F2084E28
:100DD000C5F60203C5F6000E1A6842F002021A6058
:100DE0001A6807F00C0302F002020292029A29F03C
:100DF0000302019C009E082C38BF26460F2452F89F
:100E00000EC09C402CEA040406FA03F34FF0B04CE9
:100E1000234342F80E30DCF800204B6842EA080613
:100E2000DC0258BF22EA08069C02CCF8006040F2BF
:100E3000040CC5F6000CDCF8002042EA080658BF96
:100E400022EA08069C03CCF80060DCF8802042EA25
:100E5000080658BF22EA0806DB03CCF88060DCF8FD
:100E60007C2042EA080658BF22EA0806CCF87C60DB
:100E70004EE703B0BDE8F08F40F25C10C2F20040D4
:100E8000006870470000000040F2080040F25C116A
:100E9000C2F20040C2F2004100780A6810440860C3
:100EA000704700000000000080B5032000F0A4F8A7
:100EB00000F022FF44F2184142F63063C5F6020109
:100EC000C0F600030A68096801F00F01C2F30322AB
:100ED000595C9A5C01F01F0102F01F02D04040F201
:100EE0000402C2F2004220FA01F1116040F2000156
:100EF000C2F2004108600F2000F00AF800281CBF71
:100F0000012080BD00F054F8002080BD00000000EA
:100F1000B0B58AB00F2840D804461C2000222146D4
:100F2000002500F059F81C2000F052F840F20C00A7
:100F3000C2F20040046044F2E840C5F602000168D5
:100F400041F001010160006801A900F00100029078
:100F5000029802A800F068FE079C002C18BF01242C
:100F600000F0B6FE4DF68361A040C4F21B314FF095
:100F7000FF32A0FB010140F21010C2F200404FF01E
:100F80008043036002EB9141C0E9011540F2E73173
:100F9000C0E9031501F050FA10B101200AB0B0BD4C
:100FA00040F21010C2F2004001F07AFA0AB0B0BD6F
:100FB00081B044F2F440C5F60200016841F002013C
:100FC0000160006800F002000090009801B07047D6
:100FD00080B501F0B5FE80BD70B514460D460646DD
:100FE00001F0BEFE2946224601F0EAFB01463046EA
:100FF00001F0BEFE70BD000080B501F0CDFE80BDE9
:10100000B0B544F60C05C5F60205296849072968FC
:1010100005D401F00701081A18BF0120B0BD21F066
:10102000070108432860FFF727FF044655F8080C1E
:10103000800407D4FFF720FF001BB0F57A7FF5D9B5
:101040000120B0BD0020B0BD2DE9F04381B00446C1
:10105000C07844F22C490007C5F6020901D40025E6
:101060002EE0606E4FEA305003280DD80025DFE8EF
:1010700000F0020E1714D9F80000002540F40030EB
:10108000C9F8000055B913E001253DB910E004F19D
:101090000800022101F0B0FB05464DB1A84611E061
:1010A00004F12800022101F037FC0546002DF5D19E
:1010B000D9F82400616E20F440100843C9F82400D8
:1010C0004FF000086078C00730D0A06D042807D822
:1010D000DFE800F00A131C030300FDB1A84625E079
:1010E0000125002DFAD119E0D9F8000040F40030B4
:1010F000C9F80000002DF1D110E004F10800002132
:1011000001F07AFB0546002DE8D107E004F1280044
:10111000002101F001FC0546002DDFD1D9F82400A3
:10112000A16D20F007000843C9F82400607840074B
:1011300034D5D4F8A4004FEA7050052807D8DFE86A
:1011400000F00A131C030303FDB1A84626E00125A5
:10115000002DFAD119E0D9F8000040F40030C9F8A8
:101160000000002DF1D110E004F10800002101F091
:1011700043FB0546002DE8D107E004F128000021DB
:1011800001F0CAFB0546002DDFD1D9F82C00D4F8B8
:10119000A41020F460000843C9F82C006078000710
:1011A00034D5D4F8A8004FEA3060052807D8DFE826
:1011B00000F00A131C030303FDB1A84626E0012535
:1011C000002DFAD119E0D9F8000040F40030C9F838
:1011D0000000002DF1D110E004F10800002101F021
:1011E0000BFB0546002DE8D107E004F128000021A3
:1011F00001F092FB0546002DDFD1D9F82C00D4F880
:10120000A81020F0E0600843C9F82C00E0788007BF
:1012100028D5E06C4FEA3010032806D8DFE800F04C
:1012200002091202B5B1A8461CE00125002DFAD131
:1012300010E0D9F8000040F40030C9F80000002D9B
:10124000F1D107E004F10800022101F0D5FA0546CA
:10125000002DE8D1D9F82000E16C20F030000843DF
:10126000C9F820006078C00632D5E06D4FEA303012
:10127000042807D8DFE800F00A131C030300FDB1BF
:10128000A84625E00125002DFAD119E0D9F8000083
:1012900040F40030C9F80000002DF1D110E004F155
:1012A0000800002101F0A8FA0546002DE8D107E06A
:1012B00004F12800002101F02FFB0546002DDFD1AD
:1012C000D9F82400E16D20F4E0400843C9F8240077
:1012D0006078800626D5206E4FEA3040052807D872
:1012E000DFE800F0030A100303039DB1A84619E0EC
:1012F0000125002DFAD10DE004F10800012101F0D3
:101300007BFA04E004F12800012101F005FB054609
:10131000002DEBD1D9F82400216E20F4E020084301
:10132000C9F824006078400628D5D4F8AC004FEA0C
:101330003070052807D8DFE800F0030A1003030324
:101340009DB1A8461AE00125002DFAD10DE004F167
:101350000800012101F050FA04E004F12800012105
:1013600001F0DAFA0546002DEBD1D9F82C00D4F8BB
:10137000AC1020F0E0400843C9F82C00607800066B
:1013800020D5E06ED8B1B0F1005F12D0B0F1805F2F
:1013900025D1D9F8000040F40030C9F8000085B923
:1013A000D9F82400E16E20F040500843C9F8240029
:1013B00008E004F10800012101F01EFA0546002DA5
:1013C000EED0A846E078C0072AD0A06C03280AD83F
:1013D000DFE800F0020D1602D5B1A84620E0012595
:1013E000002DEED1DCE70125002DF6D110E0D9F873
:1013F000000040F40030C9F80000002DEDD107E0F6
:1014000004F10800022101F0F7F90546002DE4D1AE
:10141000D9F82000A16C20F003000843C9F820008F
:10142000A078400642D5D9F8D40340F48070C9F8BA
:10143000D403FFF721FD0646D9F8D403C00505D42F
:10144000FFF71AFD801B6528F6D303256DBBD9F87D
:101450004410D4F8B000414011F4407F11D0D9F8C5
:101460004410D9F8442042F48032C9F84420D9F815
:10147000442021F4407122F48032C9F84420C9F894
:101480004410B0F5807F0FD1FFF7F6FC064641F21D
:10149000893700BFD9F84400800705D4FFF7ECFC7A
:1014A000801BB842F6D3032585B1A8462078C00733
:1014B00042D0A06F4FEAF000052823D8DFE800F003
:1014C00003262C0303037DB3A84635E04FF6CF7304
:1014D000D4F8B00059F81C2CC0F2FF0300F440719E
:1014E00022F47C5203EA1013B1F5407F08BF1A437F
:1014F0006FF31F3049F81C2CD9F844100843C9F881
:101500004400D3E70125002DDED10DE004F10800F1
:10151000012101F071F904E004F12800012101F03A
:10152000FBF90546002DCFD1D9F82800A16F20F096
:1015300038000843C9F828002078800724D5606F58
:10154000052807D8DFE800F0030A100303039DB164
:10155000A84619E00125002DFAD10DE004F108009C
:10156000012101F049F904E004F12800012101F012
:10157000D3F90546002DEBD1D9F82800616F20F092
:1015800007000843C9F828002078400726D5D4F87A
:101590009000052807D8DFE800F0030A10030303D2
:1015A0009DB1A8461AE00125002DFAD10DE004F105
:1015B0000800012101F020F904E004F128000121D4
:1015C00001F0AAF90546002DEBD1D9F82C00D4F88A
:1015D000901020F007000843C9F82C0020788006FE
:1015E00028D5D4F88C004FEA3070052807D8DFE8FA
:1015F00000F0030A100303039DB1A8461AE0012579
:10160000002DFAD10DE004F10800002101F0F4F8FA
:1016100004E004F12800022101F07EF90546002DC6
:10162000EBD1D9F82800D4F88C1020F0E040084322
:10163000C9F828002078400628D5D4F898004FEA49
:10164000B020052807D8DFE800F0030A10030303E1
:101650009DB1A8461AE00125002DFAD10DE004F154
:101660000800002101F0C8F804E004F1280002217C
:1016700001F052F90546002DEBD1D9F82C00D4F831
:10168000981020F4E0500843C9F82C002078000698
:1016900028D5D4F89C004FEA7030052807D8DFE839
:1016A00000F0030A100303039DB1A8461AE00125C8
:1016B000002DFAD10DE004F10800002101F09CF8A2
:1016C00004E004F12800022101F026F90546002D6E
:1016D000EBD1D9F82C00D4F89C1020F460400843DA
:1016E000C9F82C002078000716D5D4F88000B0F592
:1016F000805F08D104F12800022101F00DF90028D3
:1017000018BF4FF00108D9F82800D4F8801020F451
:1017100040500843C9F828002078C00616D5D4F8F0
:101720009400B0F5807F08D104F12800022101F077
:10173000F3F8002818BF4FF00108D9F82C00D4F8AE
:10174000941020F440700843C9F82C00A0780007DA
:1017500022D5D4F8A000B0F5003F1AD0B0F5803FF4
:1017600011D0C8BB04F10800002101F045F805467E
:101770008DB9D9F82C00D4F8A01020F440300843DB
:10178000C9F82C0008E004F12800022101F0C4F897
:101790000546002DEDD0A846A078400729D5D4F8FD
:1017A0008400B0F5401F21D0B0F5001F18D0B0F56F
:1017B000801F40F0BB80D9F8000040F40030C9F829
:1017C0000000ADB9D9F82800D4F8841020F44010F6
:1017D0000843C9F828000CE00125002DDBD1C8E73B
:1017E00004F12800012101F097F80546002DE9D009
:1017F000A846A078C00720D0206DB0F5803F10D05B
:10180000B8B9D9F8000040F40030C9F800009DB91B
:10181000D9F82000216D20F480300843C9F8200059
:101820000BE004F10800022100F0E6FF05461DB9B7
:10183000EEE70125002DEBD0A846E078800608D51C
:1018400004F12800022101F067F8002818BF4FF0CA
:101850000108D4E900108A0377D5E26F6FF0010325
:1018600003EB3223022B0AD34FEA32233BB1012B85
:1018700061D1D9F8003043F40033C9F80030002DAD
:101880005CD0CA0264D48A026CD44A0075D4B1F127
:10189000FF3F40F38380090200F18B80C00707D02F
:1018A00004F10800002100F0A7FF002818BF05463A
:1018B0002079800707D504F10800012100F09CFF82
:1018C000002818BF05462079400707D504F1080015
:1018D000022100F091FF002818BF0546207900077B
:1018E00007D504F12800002101F016F8002818BFE0
:1018F00005462079C00607D504F12800012101F032
:101900000BF8002818BF05462079800607D504F19A
:101910002800022101F000F8002818BF0125002D41
:1019200018BF0125284601B0BDE8F0830125002D30
:101930007FF45EAF46E70125002DA2D1D9F828300B
:1019400023F440731A43C9F828204546CA029AD5A1
:10195000D9F82420236F22F000421A43C9F824202A
:101960008A0292D5D9F82420A36E22F080721A43FD
:10197000C9F824204A007FF58AAF59F81C2C22F4BC
:10198000004249F81C2CD4F8B42059F81C3C1A43E6
:1019900049F81C2CB1F1FF3F3FF77DAFD9F820206B
:1019A000636D22F040521A43C9F8202009027FF5E6
:1019B00075AFD9F82810D4F8882021F440011143DC
:1019C000C9F82810C0077FF46BAF71E70000000072
:1019D0002DE9F04381B0002800F0F48042F20008C5
:1019E0000446C5F200288946D8F8000000F00F0030
:1019F00088420ED2D8F8000020F00F0040EA09001B
:101A0000C8F80000D8F8000000F00F00484540F08A
:101A1000D980206844F218474107C5F602070AD565
:101A200021693A6802F07002914204D93A6822F0C2
:101A300070021143396001070AD561697A6802F0C2
:101A40007002914204D97A6822F0700211437960E1
:101A5000C1060AD5A1697A6802F4E062914204D90C
:101A60007A6822F4E0621143796081060AD5E1695F
:101A7000BA6802F07002914204D9BA6822F070028A
:101A80001143B96081070AD5E1683A6802F00F0294
:101A9000914204D93A6822F00F0211433960C0071D
:101AA0007ED1206881070AD5E1683A6802F00F020A
:101AB000914204D23A6822F00F0211433960D8F8FB
:101AC000001001F00F0149450DD9D8F8001021F0A0
:101AD0000F0141EA0901C8F80010D8F8001001F020
:101AE0000F0149456ED141070AD521693A6802F0D4
:101AF0007002914204D23A6822F0700211433960B8
:101B000001070AD561697A6802F07002914204D235
:101B10007A6822F0700211437960C1060AD5A16982
:101B20007A6802F4E062914204D27A6822F4E062B8
:101B30001143796080060AD5E069B96801F0700147
:101B4000884204D2B96821F070010843B86000F0FF
:101B5000D3F8396842F63062C0F600023B68C1F340
:101B6000032103F00F03515CD25C01F01F01C84058
:101B700002F01F0140F2040220FA01F1C2F2004219
:101B8000116040F2000140F20C02C2F20041C2F2C8
:101B9000004208601068FFF7BBF901B0BDE8F083B0
:101BA000386820F47061D4E90102012841EA020199
:101BB00039600BD003282BD002282ED157F8181CDF
:101BC000890307D4012001B0BDE8F08357F8181C41
:101BD000C905F7D557F8081C21F00701084347F855
:101BE000080CFFF749F9064641F2883557F8080C0A
:101BF000616800F03800B0EBC10F3FF452AFFFF75F
:101C00003BF9801BA842F1D9032001B0BDE8F08365
:101C100057F8181C8901D5D5DCE757F8181C490777
:101C2000D0D5D7E7000000003F22026044F21842FE
:101C3000C5F6020252F8083C03F00703436013683C
:101C400003F470638360136803F00F03C3601368C9
:101C500003F070030361536803F07003436153683A
:101C600003F4E0638361926802F07002C26142F2A1
:101C70000000C5F20020006800F00F000860704707
:101C800080B500F039F844F2184142F63063C5F6E9
:101C90000201C0F600030A68096801F00F01C2F3EF
:101CA0000322595C9A5C02F01F0220FA02F201F052
:101CB0001F0040F2040122FA00F0C2F20041086065
:101CC00040F20001C2F200410A6080BD0000000045
:101CD00080B5FFF7D5FF44F21C4142F63062C5F6ED
:101CE0000201C0F600020968C1F30211515C01F063
:101CF0001F01C84080BD000044F20041C5F602014A
:101D00000869C0F3C20003280FD002282AD070BB94
:101D10000868800649F20000C0F2D03058BF704712
:101D20000968C1F3C101C84070478A6A886AC0F374
:101D3000051CC86ABCF1000F4B6B1DD0C3F3CC036C
:101D400000F00100584302F00302022A00EE100ADC
:101D5000B8EE400A12D0A2B90868800614D49FEDEC
:101D6000261A1EE043F20060C0F26E10704740F683
:101D70000010C0F23D007047002070479FED1D1A13
:101D80000FE09FED1B1A0CE0086849F20002C0F258
:101D9000D032C0F3C10022FA00F001EE100AB8EE12
:101DA000411A086B9FED153A6FF35F2002EE100A9F
:101DB000086BC0F34620B8EE422A013000EE032A39
:101DC00000EE10CAB7EE003AB8EE400A81EE000A03
:101DD00032EE031A20EE010A01EE100AB8EE411AA3
:101DE00080EE010ABCEEC00A10EE100A704700BF78
:101DF0000024744A001BB74B0024744C00000039C7
:101E00002DE9F04381B0F8B18046007844F20049F2
:101E1000C007C5F602095CD0D9F8100000F03801FF
:101E2000D9F82800102905D018290FD100F0030097
:101E300002280BD1D9F80000800346D5D8F8040059
:101E4000002842D1012731E00127E2E2D8F804500E
:101E50002DB1B5F5A02F0DD0B5F5803F10D0D9F834
:101E6000000020F48030C9F80000D9F8000020F408
:101E7000802009E0D9F8000040F48020C9F8000073
:101E8000D9F8000040F48030C9F80000FEF7F4FFF4
:101E9000002D054615D000BFD9F80000800314D4EA
:101EA000FEF7EAFF401B6428F6D90327002000282C
:101EB00000F0AF820DE000BFFEF7DEFF401B64289C
:101EC000F3D8D9F800008003F6D40120002800F0F0
:101ED000A08298F8000080076AD5D9F8100010F0A9
:101EE0003801D9F828001DD0182908BF5FEA807092
:101EF00018D0D8F80C00D9F80010002840D021F0F4
:101F000019010843C9F80000FEF7B6FF054600BFF7
:101F1000D9F80000400727D4FEF7AEFF401B022887
:101F2000F6D91EE0D9F80000400704D5D8F80C0017
:101F3000002800F05E81D9F80000D8F80C1020F0DD
:101F400019000843C9F80000FEF796FF054600BFD8
:101F5000D9F80000400707D4FEF78EFF401B022887
:101F6000F6D90327002420E0D9F80400D8F810108F
:101F700020F0FE40012440EA0160C9F8040014E0AA
:101F800021F00100C9F80000FEF776FF05460126A2
:101F9000D9F8000010F0040086EA900405D0FEF79E
:101FA0006BFF401B0328F3D30327002C00F0318282
:101FB00098F80000C00656D5D9F8100000F0380196
:101FC000D9F82800082905D0182917D100F00300F6
:101FD000012813D1D9F80000C00503D5D8F81C009A
:101FE00080283BD1D9F80C00D8F8201020F07C5084
:101FF000012440EA0160C9F80C0031E0D8F81C0067
:102000000028D9F8000012D040F08000C9F8000084
:10201000FEF732FF054600BFD9F80000C005E1D445
:10202000FEF72AFF401B0228F6D9032717E020F00D
:102030008000C9F80000FEF71FFF0546012600BF1B
:10204000D9F8000010F4807086EA102408D0FEF75A
:1020500013FF401B0328F3D3032701E001270024CB
:10206000002C00F0D68198F8000000071CD498F8E6
:102070000000800631D498F80000400745D4D8F815
:102080002440002C00F09180D9F8100000F03800B6
:10209000182840F08C80012CD9F82810D9F830008D
:1020A00040F0A9800127B4E1D8F814000028D9F83D
:1020B00074003ED040F00100C9F87400FEF7DCFE69
:1020C000054600BFD9F874008007D0D4FEF7D4FECF
:1020D000401B0228F6D903279BE1D8F818000028F6
:1020E000D9F800004DD040F48050C9F80000FEF748
:1020F000C3FE0546D9F800008004BCD4FEF7BCFE40
:10210000401B0228F6D9032783E1D9F8000440F4E4
:102110008070C9F80004FEF7AFFE0546D9F8000448
:10212000C0051AD4FEF7A8FE401B6428F6D9032781
:102130006FE120F00100C9F87400FEF79DFE05462E
:10214000032700BFD9F8740080077FF590AFFEF732
:1021500093FE401B0228F5D95BE1D8F808502DB159
:10216000052D00F08280012D00F08580D9F87000E7
:1021700020F00100C9F87000D9F8700020F00400C8
:102180007DE020F48050C9F80000FEF775FE05469A
:10219000032700BFD9F8000080047FF56CAFFEF77D
:1021A0006BFE401B0228F5D933E1002731E1D9F855
:1021B000000020F08070C9F80000FEF75DFE022CE0
:1021C00005464FF0030709D1D9F80000800178D502
:1021D000FEF752FE401B0228F6D91AE1D9F800009A
:1021E000800140F1E780FEF747FE401B0228F5D949
:1021F0000FE10127B6E601F00302D8F828309A4231
:1022000040F0DA80C1F30511D8F82C20914240F05B
:10221000D7800146D8F830206FF35F21013A914210
:1022200040F0D080C0F34622D8F8341001398A42F9
:1022300040F0CA80C0F30642D8F8381001398A420B
:1022400040F0C480C0F30660D8F83C1001398842E1
:1022500040F0BE80D9F83400D8F84810C0F3CC0064
:10226000814240F0B7800027D3E0D9F8700040F0F9
:102270000400C9F87000D9F8700040F00100C9F8F6
:102280007000FEF7F9FD002D054641F288344FF04D
:10229000030711D0D9F8700080073FF5F0AEFEF7C4
:1022A000EBFD401BA042F5D9B3E000BFFEF7E4FD13
:1022B000401BA04200F2AD80D9F870008007F5D431
:1022C000DDE608F12807D9F8280040F2F331884309
:1022D0008ECF0843591E40EA02104FF47E426FF33E
:1022E0005F21C9F8280002EB47204FF4FE0280B2BC
:1022F000D8F83C300844D8F8381002EB01414FF0D0
:10230000FE4201F4FE0102EB0362084402F0FE41CA
:102310000844C9F83000D9F82C004FF6F87120F0C5
:102320000100C9F82C00D9F83400D8F848208843B7
:1023300040EAC200C9F83400D9F82C00D8F840109F
:1023400020F00C000843C9F82C00D9F82C00D8F86C
:10235000441020F002000843C9F82C00D9F82C00E2
:1023600040F48030C9F82C00D9F82C0040F400303B
:10237000C9F82C00D9F82C0040F48020C9F82C00B2
:10238000D9F82C0040F00100C9F82C00D9F8000061
:1023900040F08070C9F80000FEF76EFD0446032788
:1023A000D9F80000800109D4FEF766FD001B022861
:1023B000F6D92EE000272CE001272AE0002728E0AC
:1023C000012726E0012724E0012722E0012720E061
:1023D00001271EE0D9F82C0020F00100C9F82C00DC
:1023E000FEF74AFD0546FEF747FDA842FBD0D9F8A7
:1023F00034004FF6F871D8F848208843002740EAA7
:10240000C200C9F83400D9F82C0040F00100C9F826
:102410002C00F8B201B0BDE8F0830000000000001D
:10242000704700000000000070470000000000003E
:10243000704700000000000060B310B5044690F83B
:102440003D0028B9002084F83C00204600F024F824
:10245000022084F83D002068211D00F0BDFB012012
:1024600084F8480084F83E0084F83F0084F8400077
:1024700084F8410084F8420084F8430084F8440062
:1024800084F8450084F8460084F8470084F83D004D
:10249000002010BD012070477047000000000000C0
:1024A00090F83D10012922D1022180F83D100168E9
:1024B0004DF6FF70C4F200008142C86840F0010090
:1024C000C86016DC40F2FF70C4F20000814226DDD5
:1024D00040F60000C4F20000814232D040F60040D5
:1024E000C4F2000081422CD041F6000025E001201A
:1024F00070474FF6FF70C4F20000814215DD0020E6
:10250000C4F2010081421CD044F20000C4F2010078
:10251000814216D040F20040C4F201000FE0B1F158
:10252000804F0ED040F2004007E04EF20000C4F2AF
:102530000000814205D04EF20040C4F2000081420A
:102540000BD107228868C0F2010202400020062A4F
:1025500018BFB2F5803F00D17047086840F0010015
:102560000860002070470000704700000000000075
:10257000F0B581B004460068C768066906EA070539
:10258000A90727D4680756D428076CD4E80600F1B9
:102590008280E80706D020686FF0010101612046C3
:1025A00000F09EF817F0800718BF16F4025006D00E
:1025B00020686FF4025101612046FFF735FF002FBC
:1025C00018BF16F4807011D1680618D4A8061FD45D
:1025D00001B0F0BD6FF00201016101212177806936
:1025E00080071ED02046FFF7BFFF20E020686FF471
:1025F000807101612046FFF713FF6806E6D5206869
:102600006FF040010161204600F076F8A806DFD5A2
:1026100020686FF0200101612046FFF709FF01B03B
:10262000F0BD204600F054F8204600F055F8002098
:1026300020776807A8D520686FF0040101610221A6
:102640002177806910F4407F03D02046FFF78CFF8C
:1026500005E0204600F03CF8204600F03DF8002060
:102660002077280792D520686FF0080101610421C6
:102670002177C069800703D02046FFF775FF05E08A
:10268000204600F025F8204600F026F800202077AC
:10269000E8067FF57EAF20686FF010010161082128
:1026A0002177C06910F4407F03D02046FFF75CFF1C
:1026B00005E0204600F00CF8204600F00DF8002060
:1026C0002077E8077FF467AF6CE7000000000000A8
:1026D000704700000000000070470000000000008C
:1026E00080B50068B0F1804F18BF80BDFEF7CCFB0D
:1026F00080BD0000000000007047000000000000E6
:10270000FEE700000000000080B540F270004AF2D1
:102710000001C2F20040C4F200014FF0010C4FF082
:10272000030E01600021C0E9021101820A2280F833
:1027300012C01D23C0F814E08261C0E90732C0E96D
:1027400009E2C0E90B32C0E90D1CC1630422C0E9F3
:102750001022C0E91212C0E91412C0E91611C0E932
:1027600018218266FEF724F9002808BF80BDFDF716
:102770008FFE80BD0000000082B044F2E040C5F64C
:102780000200016841F080010160016801F08001F0
:1027900001910199016841F008010160006800F0B1
:1027A00008000090009802B0704700000000000090
:1027B000FEE7000000000000FEE70000000000004F
:1027C00000F007004FF0FF3C80F00703042B28BF08
:1027D0000423033838BF00200CFA03F399430CFAA2
:1027E00000F301FA00F022EA0301084370470000F9
:1027F0007047000000000000F0B581B044F22C47A3
:10280000C5F6020757F8042C02F00302032A02D18E
:10281000012001B0F0BD054657F82C0C0C4620F005
:10282000806047F82C0CFEF727FB064657F82C0C67
:10283000000105D5FEF720FB801B0228F6D964E0D5
:1028400057F8040CEE6895E80E0020F47C30012C5B
:1028500040EA0130A2F101016FF35F214FF47E42A3
:1028600002EB432247F8040C92B24FF0FE4302EB16
:1028700001004FF4FE012A6901EB064101F4FE015B
:1028800003EB0262084402F0FE410844F860386835
:10289000696920F0C00040EA010038603868A96921
:1028A00020F0200040EA0100386038684FF6F871E7
:1028B00020F0100038603869EA6920EA01004FF41E
:1028C000001140EAC2003861386808BF4FF4801137
:1028D00040F01000002C386008BF4FF40021386829
:1028E0000843386057F82C0C40F0806047F82C0CF7
:1028F000FEF7C2FA044600BF57F82C0C000107D4BB
:10290000FEF7BAFA001B0328F6D3032001B0F0BD8E
:10291000002001B0F0BD0000F0B581B044F22C47BA
:10292000C5F6020757F8042C02F00302032A02D16D
:10293000012001B0F0BD054657F82C0C0C4620F0E4
:10294000805047F82C0CFEF797FA064657F82C0CE7
:10295000800005D5FEF790FA801B0228F6D964E0C6
:1029600057F8040CEE6895E80E0020F07C70012CFE
:1029700040EA0150A2F101016FF35F214FF47E4262
:1029800002EB432247F8040C92B24FF0FE4302EBF5
:1029900001004FF4FE012A6901EB064101F4FE013A
:1029A00003EB0262084402F0FE4108447861386893
:1029B000696920F4406040EA010038603868A9691C
:1029C00020F4007040EA0100386038684FF6F87172
:1029D00020F480703860B869EA6920EA01004FF09D
:1029E000807140EAC200B861386808BF4FF4000146
:1029F00040F48070002C386008BF4FF480013868C4
:102A00000843386057F82C0C40F0805047F82C0CE5
:102A1000FEF732FA044600BF57F82C0C800007D4AA
:102A2000FEF72AFA001B0328F6D3032001B0F0BDFD
:102A3000002001B0F0BD0000704700000000000061
:102A40007047000000000000B0B59CB044F61804C8
:102A500009A84C21C5F60204FDF7ACFC02200025B4
:102A6000CDE90755CDE90555CDE90355CDE901552A
:102A7000FEF7C6FA0095206820F4404020602068E8
:102A800000F440400090009820688004FCD50120AC
:102A900009904FF480310A9102212822CDE91520B6
:102AA00004201491CDE917010C20199009A80024E5
:102AB000CDE91211CDE91A44FFF7A2F9A8B93F20D8
:102AC000019003204FF48061CDE9020408200490B6
:102AD0004020CDE90500CDE9071001A80321FEF74C
:102AE00077FF002804BF1CB0B0BDFDF7D1FC00008B
:102AF0004EF6885042F2000CCEF20000C5F2002CD7
:102B0000026842F470020260DCF8000000F00F007E
:102B1000062806D8DCF80000072262F30300CCF890
:102B2000000044F200404EF67F51C5F60200CEF69A
:102B3000F621026842F0010202600022026103688D
:102B400019400160DCF80010090706D5DCF8001018
:102B5000072363F30301CCF8001040F200218261E7
:102B6000C261C0F20221026281620021C0F2FF1143
:102B7000C16240F28021C0F20111016342638163AE
:102B8000C26301644264016821F48021016002662D
:102B9000D0F8D410C90448BF7047D0F8D41043F21D
:102BA000D20241F48051C0F8D41044F20001C5F2C1
:102BB00000210A60D0F8D41021F48051C0F8D4105C
:102BC000704700000000000080B540F21010C2F213
:102BD0000040FFF7CDFC80BD10B540F6FF32D0F8C5
:102BE00000E0C4F2000290420FDCB0F1804F1DD033
:102BF00040F20043C4F20003984217D040F60003AD
:102C0000C4F20003984211D015E040F60043C4F22C
:102C1000000398420AD040F20043C4F201039842F4
:102C200004D00023C4F20103984204D12EF07002B4
:102C30004B6843EA020E4EF2FF3343F6FF7CC4F2C8
:102C40000003C4F2010C98420FDD604522DC4EF215
:102C50000043C4F20003984238D00023C4F20103B9
:102C6000984233D040F2004322E040F2FF73C4F2B6
:102C70000003984221DD40F60003C4F200039842AD
:102C800024D040F60043C4F2000398421ED04EF216
:102C9000000317E044F20003C4F20103984215D088
:102CA00044F60003C4F2010398420FD044F20043FB
:102CB000C4F20103984209D00DE0B0F1804F05D075
:102CC00040F20043C4F20003984204D12EF4407253
:102CD000CB6843EA020E4B6960450A688C68C4629F
:102CE00082620EDD44F20002C4F20102904213D06F
:102CF00044F60002C4F2010290420DD044F20042B8
:102D000006E00022C4F20102904205D040F20042E7
:102D1000C4F20102904201D109690163016841F0E6
:102D200004010160012141612EF08001194301601D
:102D300010BD000000000000FEE7000000000000E1
:102D4000002848BF704700F01F01012202FA01F17C
:102D50004EF200124009CEF2000242F820107047F5
:102D60004EF60C50CEF200000068C0F3022070470F
:102D70004EF6145300F00F02CEF20003B0F1FF3F05
:102D80001A4400F16043C8BF03F5644208011070A3
:102D900070470000000000004EF60C514FF6FF0394
:102DA000CEF200010A681A4060F30A2242F0806005
:102DB00040F0FD7008607047FEF776F8FFF744FEBC
:102DC000FFF7DAFCFFF7A0FCFEE7F1EE100A4FF682
:102DD000FF71C0F2C03120EA010040F04070E1EE26
:102DE000100A704700000000000000000000000012
:102DF00000000000000000000100000002000000D0
:102E000003000000040000000000000005000000B6
:102E100000000000000000000000000006000000AC
:102E2000000000000000000000000000070000009B
:102E30000000000001020304010203040607080960
:102E4000602E0008000000241000000008030008A5
:102E5000702E000810000024500700002403000812
:102E60000090D0030090D00301000000100000008B
:04000005080002CD20
:00000001FF
